:06000000020DF002006B8E
:03000B0002006B85
:0300130002006B7D
:03001B0002006B75
:0300230002006B6D
:03002B0002006B65
:0300330002006B5D
:03003B0002006B55
:0300430002006B4D
:03004B0002006B45
:0300530002006B3D
:03005B0002006B35
:0300630002006B2D
:01006B003262
:0900800002006B0002006B00029B
:08008900006B0002006B000295
:08009100006B0002006B00028D
:08009900006B0002006B000285
:0800A100006B0002006B00027D
:0800A900006B0002006B000275
:0700B100006B0002006B0070
:0901000002006B0002006B00021A
:08010900006B0002006B000214
:08011100006B0002006B00020C
:08011900006B0002006B000204
:08012100006B0002006B0002FC
:08012900006B0002006B0002F4
:08013100006B0002006B0002EC
:08013900006B0002006B0002E4
:08014100006B0002006B0002DC
:08014900006B0002006B0002D4
:08015100006B0002006B0002CC
:08015900006B0002006B0002C4
:08016100006B0002006B0002BC
:08016900006B0002006B0002B4
:08017100006B0002006B0002AC
:07017900006B0002006B00A7
:030DF600020DFEED
:030E1100020DF9D6
:050DF9001203F180FE71
:06018000C200E4F508F5E1
:0401860009F50AD29B
:05018A0001750B00757A
:06018F000C001206001234
:0E01950005FD75CB6375CAC0758E0075C80474
:0701A300D2AFD2B0D2B122AD
:0B01AA00AA82850C827583E0EAF00554
:0501B5000C0509E4B592
:0401BA000902050A27
:0101BE00221E
:0401BF0020000122F9
:0E01C3001205FC90E6A2E0FA30E103020257BA
:0A01D100E509450A60687AC07BE783
:0E01DB008B9D7AC07BE77B008A9E90E67C7449
:0C01E90031F07460F0C3743E9509E49599
:0A01F5000A50107A3EE50924C2F515
:0601FF0009E50A34FFF5DA
:030205000A800765
:06020800AA09E4F509F566
:01020E000AE5
:0B020F008A037C007DE08D9A850B9B2C
:0E021A008A041AEC601090E67BE090E67CF01F
:080228007C007DE08D9A80EA64
:0C023000859B0B0090E68F74022BF0D22F
:03023C00CF801858
:0E023F0030CF1590E7C07431F090E7C17460C5
:0A024D00F00090E68F7402F0C2CFBB
:06025700E5AA30E00122DF
:0A025D00C3E50994C1E50A940040CE
:02026700012272
:0E02690090E690E0FB7A0090E691E0FC7D00CC
:0A027700EA4CF50DEB4DF50E7C008E
:0E0281007DF08D9A7C007DF08C9B7C007D00D2
:0A028F00C3EC950DED950E4003023F
:02029900036AF6
:07029B00E5087003020326D1
:0A02A200E50DC39CFEE50E9DFFA8CC
:0C02AC00087900C3E89EE99F5004880612
:0202B8008907B4
:0A02BA008E00E508C398F508EE2C4D
:0B02C400FCEF3DFD30012C8E008F018F
:0902CF008802890318B8FF011927
:0E02D800EA4B60B390E67BE0F582C004C005FF
:0E02E600C000C001120637D001D000D005D0F4
:0302F4000480D8AB
:0402F7008E028F03E1
:0902FB008A068B071ABAFF011BE9
:0E030400EE4F608790E67BE0F582C002C003FA
:0E031200C004C0051206741201AAD005D00462
:06032000D003D00280D5DD
:0D03260090E67BE0FA23235401FBB40100B4
:0A0333009201EA30E707743F5AF523
:03033D0008802213
:0C03400030010F8A82C004C00512060BB9
:06034C00D005D004801072
:0E0352008A82C004C0051206291201AAD00535
:02036000D004C7
:050362000CBC00010DC0
:0303670002028F00
:08036A000090E6917480F0227E
:0E03720090E6B8E0FA20E70C90E6B9E07002E1
:02038000D200A9
:04038200758201225D
:0E03860090E6B9E0FABA902B90E6BCE025E0D4
:0A039400547FFA2400F582E43418C7
:0C039E00F583E0FB90E740F0EA04240047
:0C03AA00F582E43418F583E0FA90E74196
:0303B600F0800CC8
:0C03B90090E7407436F090E7417483F048
:0D03C50090E68AE4F090E6BEE0FABA02008D
:0903D200500790E6BEE0FA80023B
:0203DB007A02A4
:0903DD0090E68BEAF07582012222
:0603E6003002031209536E
:0503EC001201BF80F5C5
:0E03F100C2AF90E609E4F01201801206C312BA
:0603FF000455120D23124B
:0804050008BDD2AF1207CC02C2
:02040D0003E604
:0A040F00AA82E50F54FEFBB50F02B0
:02041900802938
:0A041B008A048C05E46210ED621102
:0A042500EB2400F582E43418F5839F
:0A042F00E0FB7C006210EC6211E5B6
:060439001033C51133C5AC
:05043F001192E0F51030
:06044400AB0F050FEB24D5
:0A044A0000F582E43418F583EAF0AF
:010454002285
:07045500750F007510AA7578
:0C045C0011AA75820012040F75820012B4
:04046800040F7A0003
:0C046C00C3EA648094865017EA2408F567
:0C04780082E434E1F583E0F582C002125A
:07048400040FD0020A80E121
:02048B007A00F5
:0C048D00C3EA648094825017EA2423F52F
:0C04990082E434E1F583E0F582C0021239
:0704A500040FD0020A80E100
:0E04AC0075821C12040F75820012040F7A0074
:0C04BA00C3EA648094825017EA2402F523
:0C04C60082E434E1F583E0F582C002120C
:0704D200040FD0020A80E1D3
:0C04D9007486250FFAF582C00212040F91
:0C04E50090E196E0F58212040FD0029026
:0D04F100E196E02AFAF582C00212040F9095
:0B04FE00E1B4E0F58212040FD0029080
:0A050900E1B4E02AF58212040F901D
:0A051300E1DEE0F58212040F7A0029
:0E051D0090E196E0FBC3EA64808BF063F0800F
:0B052B0095F05017EA2496F582E434A6
:0C053600E1F583E0F582C00212040FD052
:04054200020A80D752
:020546007A0039
:0E05480090E1B4E0FBC3EA64808BF063F080C6
:0B05560095F05017EA24B4F582E4345D
:0C056100E1F583E0F582C00212040FD027
:04056D00020A80D727
:020571007A000E
:0E05730090E1DEE0FBC3EA64808BF063F08071
:0B05810095F05017EA24DEF582E43408
:0C058C00E1F583E0F582C00212040FD0FC
:04059800020A80D7FC
:02059C007A00E3
:0C059E00C3EA648094845017EA240EF530
:0C05AA0082E434E1F583E0F582C0021227
:0705B600040FD0020A80E1EE
:0C05BD007482250F400875820012040FA4
:0205C90080F2BE
:0805CB00AA1090187EEAF0AAC4
:0705D3001190187FEAF022ED
:0805DA007880E84400600C7910
:0C05E20001901800E4F0A3D8FCD9FAD076
:0E05EE0083D082F6D8FDC082C08375820022C1
:02E1000012010A
:06E10200000200000040D5
:06E10800C016EF03040045
:04E10E000102030106
:0AE112000A060002FFFFFF400100B3
:07E11C0009022E00010100C1
:0EE1230080FA0904000004FFFFFF02070581D7
:0EE131000200020007050202000200070504BA
:0BE13F0002000200070586020002003B
:0EE14A001201000200000040C016EF030400A6
:04E1580001020301BC
:0AE15C000A060002FFFFFF40010069
:0EE166000902200001010080FA0904000002F5
:0EE17400FFFFFF0207058102400000070502C1
:04E182000240000057
:01E186000494
:02E1870090E125
:02E1890096E11D
:02E18B00B4E1FD
:02E18D00DEE1D1
:06E1900006030000090473
:0EE196001E037700770077002E0072006500F0
:0EE1A400740072006F00310031002E00640024
:02E1B200650006
:0EE1B4002A036E0065007800790073003200C7
:0EE1C2005F006A007400610067005F003200B9
:0EE1D0006600690066006F005F006900630072
:0EE1DE001203300030003000300030003000FE
:04E1EC0030003000CF
:0105FC0022DC
:0105FD0022DB
:0105FE0022DA
:0105FF0022D9
:0B060000D2B775B5809001F4020DDF49
:0E060B00AA82ABB574FE5BF5F0741C45F0F5E9
:0E061900B5EA1392B4EAA2E192B3EAA2E49227
:02062700B222FD
:0E06290012060BA2B0E433FA74024AF58222E4
:0E063700E5821392B2D2B413C2B492B2D2B41E
:0E06450013C2B492B2D2B413C2B492B2D2B401
:0E06530013C2B492B2D2B413C2B492B2D2B4F3
:0E06610013C2B492B2D2B413C2B492B2D2B4E5
:05066F0000C2B42222CC
:0E067400E582A2B01392B2D2B4C2B4A2B01307
:0E06820092B2D2B4C2B4A2B01392B2D2B4C239
:0E069000B4A2B01392B2D2B4C2B4A2B013920C
:0E069E00B2D2B4C2B4A2B01392B2D2B4C2B4FB
:0E06AC00A2B01392B2D2B4C2B4A2B01392B2F2
:0906BA00D2B400C2B4F582222280
:0D06C30090E6007412F090E60174A3F09030
:0E06D000E6707480F00090E60274E0F0009096
:0E06DE00E60374F9F00090E6047480F00090DA
:0D06EC00E60B7403F00090E610E4F00090BF
:0D06F900E61174A0F00090E618E4F0009007
:0E070600E6047402F00090E61274A2F0009077
:0E071400E61374A2F00090E61474E0F000907A
:0E072200E6157402F00090E6047404F00090F6
:0E073000E6047406F00090E6047408F00090F1
:0E073E00E604E4F00090E60BE4F00090E649DB
:0E074C007484F00090E6497484F00090E61981
:0E075A00E4F00090E6197410F00090E632749E
:0E07680080F00090E6337404F00090E61A74FE
:0E0776000CF00090E6247402F00090E625E4FA
:0E078400F00090E6347419F00090E63574FC35
:0E079200F00090E61BE4F0000090E691748009
:0A07A000F00090E6917480F0002252
:0807AA0090E6A0E04401F022FA
:0E07B200AA8274805AC423541FFB740F5A90FD
:0C07C000E6834BF090E683E04420F0223A
:0E07CC0090E680E0440AF09000FA120DDF90F3
:0E07DA00E65D74FFF090E65F74FFF05391EF60
:0807E80090E680E054F7F022D6
:060E0B00E478FFF6D8FDBB
:060DF000751200751300EE
:0A07F00090E680E0FA30E719751476
:0307FA0000751572
:0307FD00E175168D
:0308000012751757
:03080300E1751884
:030806001C751945
:03080900E1751A7C
:03080C0066751BF3
:02080F00E122E4
:0408110075144A759B
:0308150015E17575
:03081800165C75F6
:03081B0017E1756D
:03081E00186675E4
:0308210019E17565
:030824001A1C7526
:030827001BE122B0
:09082A005391EF75A100D20232D6
:0C083300C021C0E0C0F0C082C083C00241
:0E083F00C003C004C005C006C007C000C00151
:0E084D00C0D075D0005391EF75A1001207F0D6
:0E085B00D0D0D001D000D007D006D005D004F8
:0D086900D003D002D083D082D0F0D0E0D0F8
:0208760021322D
:0C087800C021C0E0C0F0C082C083C002FC
:0E088400C003C004C005C006C007C000C0010C
:0E089200C0D075D0005391EF75A1001207F091
:0E08A000D0D0D001D000D007D006D005D004B3
:0D08AE00D003D002D083D082D0F0D0E0D0B3
:0208BB002132E8
:0508BD001207F0751C9C
:0308C2002A751D77
:0808C50008758200120C7C751D
:0308CD001C337564
:0608D0001D0875821012E4
:0408D6000C7C751C05
:0308DA0078751D11
:0C08DD0008758214120C7C90E65C7431EB
:0208E900F022FB
:0D08EB00E582547FFA24F750047582002244
:0708F800BA01047582012220
:0808FF00530201E4BA000104F8
:03090700F5822254
:0E090A00AA82BA010C90E6A1E0FB7C008B8271
:030918008C8322AB
:0E091B00BA810C90E6A2E0FB7C008B828C83FC
:0109290022AB
:0E092A0053027FEA700C90E6A0E0FB7C008B8D
:04093800828C832208
:0E093C0090E6A3E0FB7C00EAC313FA7D00EA1C
:09094A002BFBED3C8B82F58322AE
:0C095300C20290E6B8E0FA530260BA005D
:03095F00028028EB
:05096200BA2002800D27
:05096700BA4002800E01
:05096C00BA60028003E7
:03097100020C1164
:060974001207AA020C119B
:0A097A00120372E5826003020C1103
:060984001207AA020C118B
:0D098A0090E6B8E0FA530280BA80028003C4
:03099700020B123E
:0B099A0090E6B9E0FABA0003020A8BF5
:0509A500BA06028035D6
:0509AA00BA08028008FC
:0509AF00BA0A028017E6
:0309B400020B0C27
:0C09B70090E740E512F090E68AE4F09032
:0809C300E68B7401F0020C1137
:0C09CB0090E740E513F090E68AE4F0901D
:0809D700E68B7401F0020C1123
:0A09DF0090E6BBE0FABA01028017AF
:0509E900BA0202803893
:0509EE00BA030280596C
:0509F300BA0602801BA2
:0509F800BA0702803C7B
:0309FD00020A8566
:0A0A0000AA14AB1590E6B3EBF07BEF
:090A0A000090E6B4EAF0020C11C0
:0A0A1300AA16AB1790E6B3EBF07BD8
:090A1D000090E6B4EAF0020C11AD
:0A0A2600AA18AB1990E6B3EBF07BC1
:090A30000090E6B4EAF0020C119A
:0A0A3900AA1AAB1B90E6B3EBF07BAA
:090A43000090E6B4EAF0020C1187
:0E0A4C0090E6BAE0FA90E186E0FBC3EA9B4038
:070A5A00061207AA020C11AD
:0C0A610090E6BAE075F002A42487F5824C
:0B0A6D0074E135F0F583E0FAA3E0909F
:0D0A7800E6B3F07B0090E6B4EAF0020C114A
:060A85001207AA020C1189
:0D0A8B0090E6B8E0FA53021FBA0002800A9C
:050A9800BA0102801B01
:050A9D00BA0266802C86
:0E0AA20090E740E4F090E741F090E68AF09093
:080AB000E68B7402F0020C1148
:0E0AB80090E740E4F090E741F090E68AF0907D
:080AC600E68B7402F0020C1132
:0E0ACE0090E6BCE0F5821208EBE58260259010
:0E0ADC00E6BCE0F58212090AE0FA530201902E
:0E0AEA00E740EAF090E741E4F090E68AF090F1
:080AF800E68B7402F0020C1100
:060B00001207AA020C110D
:060B06001207AA020C1107
:060B0C001207AA020C1101
:0C0B120090E6B9E0FA24F45003020C0E47
:070B1E00EA2A2A900B25735F
:070B2500020C0E020B5B0243
:060B2C000BD6020BB7021C
:060B32000C0E020C0E0285
:060B38000C0E020C0E027F
:060B3E000C0E020B49023F
:050B44000C0E020B5233
:090B490090E6BAE0F512020C116D
:090B520090E6BAE0F513020C1163
:0D0B5B0090E6B8E0FA53021FBA00028005D0
:050B6800BA0247800AFB
:0A0B6D0090E6BAE01207AA020C118C
:0D0B770090E6BAE0703090E6BCE0F5821226
:0D0B840008EBE582602390E6BCE0F58212EC
:0E0B9100090AAA82AB83E0FC5304FE8A828B21
:0E0B9F0083ECF090E6BCE0F5821207B28064B1
:050BAD001207AA805FA1
:050BB2001207AA805AA1
:0E0BB70090E6B8E0FA53021FBA004F90E6BA7B
:070BC500E0FABA010280050D
:050BCC00BA02028040A6
:050BD1001207AA803BA1
:0E0BD60090E6BAE0FA702C90E6BCE0F58212D0
:0D0BE40008EBE582601A90E6BCE0F5821295
:0E0BF100090AAA82AB83E0FC4304018A828BCE
:050BFF0083ECF0800D05
:050C04001207AA8008A0
:050C09001207AA8003A0
:030C0E001207AA20
:080C110090E6A0E04480F0220F
:050C1900AA82BA0300ED
:070C1E004005EA249C50018F
:010C250022AC
:090C2600740F5AFBBB03028007A6
:070C2F00740F5AFBBB0B45DB
:0A0C3600A2AF9203C2AFEA2400F55A
:0C0C400082E43400F5837402F07B007441
:0C0C4C00012AFCE43BFDEC2400F582EDE5
:0A0C58003400F583E51DFCF0740282
:0C0C62002AFAE43BFBEA2400F582EB34A4
:0A0C6E0000F583AA1C7B00EAF0A247
:030C78000392AF35
:010C7B002256
:080C7C00E582FA2483500122F5
:060C8400EA5403600122A6
:0A0C8A00A2AF9204C2AFEA2400F505
:0C0C940082E43401F5837402F07B0074EC
:0C0CA000012AFCE43BFDEC2400F582ED91
:0A0CAC003401F583E51DF074022AFF
:0B0CB600FAE43BFBEA2400F582EB347B
:080CC10001F583AA1CEAF0A270
:040CC9000492AF22C0
:050CCD00AA82BA8000BC
:070CD2004005EA244B50012C
:010CD90022F8
:060CDA00EA540360012250
:0A0CE000A2AF9205C2AFEA2480F52E
:0C0CEA0082E43400F5837402F07B007497
:0C0CF600012AFCE43BFDEC2480F582EDBB
:0A0D02003400F583E51DF074022AA9
:0B0D0C00FAE43BFBEA2480F582EB34A4
:080D170000F583AA1CEAF0A21A
:040D1F000592AF2268
:080D2300C2E8C2EA751C00756C
:060D2B001D017582431258
:040D31000C19751C08
:030D350080751DA9
:0C0D380000758253120C190090E650E484
:0E0D4400F00090E652E4F00090E654E4F00077
:0E0D520090E656E4F00090E65174FFF0009039
:0E0D6000E65374FFF00090E65574FFF000902B
:0E0D6E00E65774FFF00090E658E4F090E65966
:0E0D7C0074FFF090E65AE4F090E65B74FFF02E
:0E0D8A0090E65CE4F090E65D74FFF090E65EAB
:0E0D9800E4F090E65F74FFF00090E660E4F097
:0D0DA6000090E66174FFF090E662E4F090CA
:0E0DB300E66374FFF090E665E4F090E6687485
:0A0DC1000BF05391AFD2E8D2EA2202
:010DCB002205
:020DCC00AA82F9
:060DCE00120DCBDAFB223E
:030DD40090FB5041
:080DD700A3E582458370F922B7
:040DDF00AA82AB83B6
:080DE300120DD41ABAFF011B26
:050DEB00EA4B70F42248
:030DFE00758121DB
:0A0E01001205DAE5826003020DF924
:00000001FF
